:06F000000C9461780C94F1
:10F0060000780C9400780C9400780C9400780C949A
:10F0160000780C9400780C9400780C9400780C948A
:10F0260000780C9400780C9400780C9400780C947A
:10F0360000780C9400780C9400780C9400780C946A
:10F0460000780C9400780C9400780C9400780C945A
:10F0560000780C9400780C9400780C9400780C944A
:10F0660000780C9400780C9400780C9400780C943A
:10F0760000780C940078626F6F746C6F61646572CF
:10F08600000053442063617264204F4B00005344D8
:10F096002063617264204552524F520040000000C6
:10F0A60000950B0035077CF00B00400788F00E003A
:10F0B6004B0794F006005907A2F00000F894EE27DB
:10F0C600EFBBF1E0F5BFF2E0F5BFF8E1A895A4B714
:10F0D600A77FA4BFF0936000E0936000E8EAF0EF3A
:10F0E60085919591009761F0A591B5910590159040
:10F0F600BF01F00105900D920197E1F7FB01F0CFFA
:10F10600EFEFEDBFE0E1EEBFC0E0D5E00C94557C3B
:10F11600AA93E881EEBDEDB5E078E9F39AC11A93BA
:10F1260010E0EFEFEEBDEDB5E078E9F31EB576C180
:10F13600BA93AA930E94E77F1FEF00E02C9AAFEFE5
:10F14600E7DF2C9830E0363048F4AC81BD81ED9194
:10F15600AC83BD83AE2FDCDF3F5FF5CF1F3F31F4BD
:10F16600DEDF1E2FA02F0F5FA536C0F3E12F0E9412
:10F17600EE7F33C1BA93AA931A930A93AE81BF81E5
:10F18600D7DFE03019F0198108818AC3C8DFEE3F66
:10F19600E9F700E010E0EA81FB810E171F0778F41B
:10F1A600EC81FD813196EC83FD833197FF93EF93DC
:10F1B600B6DFAF91BF91EC930F5F1F4FECCFAFDF80
:10F1C600AEDF2C9A198108816BC30E94DB7F2697DC
:10F1D600E1E5E883E0E0E983EA83EB83EC83EFEFA4
:10F1E600ED83AE81BF8188859985E9E00E943B7FEA
:10F1F600EE83FF83688779870E94757EE070F070E2
:10F2060060707F7FDF01CB01E8E10E94477FE983E1
:10F216000E94757EE070F0706F7F70700E94657F4F
:10F22600EA830E94757EE070FF7F60707070DF0178
:10F23600CB01E8E00E94477FEB83FE01FA93EA9355
:10F24600E3E3F5E0FA93EA93A0E0B2E093DFE0E0CF
:10F2560017C20E94E57F20E030E02C9A00E010E023
:10F266000031E0E01E0728F4AFEF52DF0F5F1F4FBB
:10F27600F7CFA9E5B7E05CDFE13069F0D9012F5F90
:10F286003F4FA53FE1E0BE0710F0E1E0A4C085E3F3
:10F296008A95F1F7EECF20E030E0E1E4E0935907FC
:10F2A600EFEFE0935E07A9E5B7E042DFE03061F0FB
:10F2B600D9012F5F3F4FA93EE3E0BE0710F0E2E021
:10F2C6008AC00E947A7EEFCF2C9AA0E0B0E080E060
:10F2D60090E07BDFA0913107A53521F4A09132079C
:10F2E600AA3A11F0E3E077C0A0913305AB3E21F4D2
:10F2F600A0913505A03909F007C0E0E0F0E0E09301
:10F306000805F093090507C0A8E0B5E0E091F90605
:10F31600F0E0ED93FC93A0910805B09109058827CC
:10F32600992753DFA0913107A53521F4A091320723
:10F33600AA3A11F0E4E04FC043E355E0FA01E5854F
:10F34600E0930105FA01A685B785E0910805F091DD
:10F356000905EA0FFB1FE0930A05F0930B05FA0176
:10F3660000881124DA0156960E94BD7FD0010E94C2
:10F376006F7FE0930C05F0930D05A0910A05B091FF
:10F386000B05E0910C05F0910D05EA0FFB1FE093CC
:10F396000205F0930305E0E0F0E0E0930405F09346
:10F3A6000505FA01A189B289E0E2F0E00E946F7FCB
:10F3B6000F01DA011B960E94BD7FD0010E94977F44
:10F3C600A0910205B0910305EA0FFB1FE093060525
:10F3D600F0930705E0E00E94EC7F269608951A93C5
:10F3E60010E8E7E0E7B95E9A0E947A7E103898F056
:10F3F6005C9A0E947A7EE6B1E07F1E2F5C980E949E
:10F406007A7E5C9A0E947A7EE6B1F0E00E945C7F8A
:10F416001E0F5C98EBCFE7EFE7B95E98E12F1991E5
:10F42600089585E38A95F1F75C9A85E38A95F1F765
:10F436005C9885E38A95F1F70895AA93D0DFE88171
:10F44600E07F0E947E7EE881E295E07F0E947E7EDC
:10F456005F9821960895BA93AA931A9310E0A9810A
:10F46600BA81EE27A10FBE1FEC91E03049F0A981C9
:10F47600BA81EE27A10FBE1FAC91DFDF1F5FEFCF72
:10F48600188123960895AA931A93A9DFE981E07F4C
:10F496001E2F136018B9C5DFE981E295E07F1E2FA4
:10F4A600136018B9BEDF18810C945A7E1A930A931A
:10F4B60010E00FEFE7E0E7B9083014F4103009F078
:10F4C60011C00F5FE02FE86FE8B9AAE0B0E00E9434
:10F4D600237FE6B1E877F0E00E94607F1E2FEEE121
:10F4E6001E27EACF103011F4E0E027C00770043081
:10F4F6001CF40150100F0BC00370103109F41CE00E
:10F50600123009F410E0E02FE10FE0681E2FE3E06F
:10F51600E8B912C01A930A9310E000E0011711F43B
:10F52600003029F4C3DF0E2FC1DF1E2FF7CF0030C6
:10F5360019F0BCDF0E2FFBCFE12F09911991089529
:10F54600BA93AA9324971A930A93289A29982A9ADF
:10F55600E0910205F091030566277727EA83FB838E
:10F566006C837D83E885F985AA81BB818C819D8129
:10F57600662777270E94327FE0910405F091050502
:10F586000E948B7EEA83FB836C837D83AA81BB8189
:10F596008C819D811ADEEE81FF81ED5CFA4F8F0131
:10F5A600D801EC91E03011F40C943B7BF801A38573
:10F5B600AF3021F0D801AC91A53E09F456C0F80150
:10F5C600A085A83431F4A185A53419F4A285A835FF
:10F5D60009F048C0F801A28DB38D12970E94907E63
:10F5E6000E946F7FDF010E94947EEA0FFB1FE0936B
:10F5F6003307F0933407E0E0E0930E05E0930F0540
:10F606000E94997ED8015A960E94BD7FE09312050A
:10F61600F0931305E0E0F0E060E070E0E0931C0595
:10F62600F0931D0560931E0570931F05E093160564
:10F63600D8015C960E94C17FE0931805F0931905E6
:10F6460060931A0570931B05A4E91DDFD8011B966C
:10F65600E0E0EC93D801FFDE2898299A2A9AE0E0A8
:10F66600F0E00CC0E1E0F0E009C0E1E0F0E006C047
:10F67600E0E2F0E05E2E6F2EE2E0F0E01981088114
:10F686002A960895AA930E94E57FAE81A23018F1CA
:10F69600B0E0E0E0F1E00E94AA7FAF01E0910A0548
:10F6A600F0910B05E40FF51F8F01D80188279927E4
:10F6B6008CDDAE81E2E0EA9FF001DF01ED5CFA4FFE
:10F6C60060817727FD01EC5CFA4FF081E0E0E60F00
:10F6D600F71F9F0102C02FEF3FEFF9010E94EC7F59
:10F6E6002796089524971A93E0911005F091110535
:10F6F600ED5CFA4F1081A0E1B5E0ED91FD913196F8
:10F70600FE93EE93ACE1B5E00E94C77FEF5FFF4F3B
:10F716006F4F7F4F0E94CC7FA0911C05B0911D05B5
:10F7260080911E0590911F05E0911805F09119052D
:10F7360060911A0570911B050E94E07F90F4ACE180
:10F74600B5E00E94C77F3197604070400E94CC7F31
:10F75600EF5FFF4F6F4F7F4FE1E0E0931605E0E06C
:10F766004DC0A0911005B0911105A030E2E0BE0792
:10F7760010F40C94007CAEE0B5E0ED91FD9131966D
:10F78600FE93EE93E0910105A0910E05B0910F0551
:10F79600F0E0AE17BF0760F0A091120573DFE093AB
:10F7A6001205F0931305E0E0E0930E05E0930F05D4
:10F7B6000E94A07E0E94A87E0E94907E0E94AD7E3E
:10F7C6000E946A7F0E94777F0E94A87E0E94947E94
:10F7D6000E94AD7E0E948B7E0E94A87EE0910E055F
:10F7E600F0910F050E94AD7E0E948B7E0E94A87E3E
:10F7F6000E94AD7EEADC0E94997EE12F1881259653
:10F806000895BA93AA930E94E57F00E010E02E8146
:10F816003F8150E0543010F00C94507C0E94B27E30
:10F82600A03320F00E94B27EAA3308F004C00E94E2
:10F83600B87EE053EC930E94B27EA13420F00E9481
:10F84600B27EA73408F004C00E94B87EE753EC935A
:10F85600503049F40E94BF7EF0E00E94537FFE2F95
:10F86600E0E00E0F1F1F513031F40E94BF7EFE2FC5
:10F87600E0E00E0F1F1F523039F40E94BF7EF0E009
:10F886000E94537F0E0F1F1F533029F40E94BF7E24
:10F89600F0E00E0F1F1F5F5FBDCFF8010E94EC7FE7
:10F8A600289608952497EBEFE5B9EFEBE4B9EFEF6F
:10F8B600E8B9E3EFE7B9E0E2EBB9E0EFEAB9E0E592
:10F8C600ECBDE0E0EDBD0E945C7E289A299A2A985C
:10F8D600A8EEB3E00E94237FE0E3E8B900E003303E
:10F8E60038F49FDDA9E1B0E00E94237F0F5FF7CFD8
:10F8F60076DDE0E2E8B995DD72DDA8E2C4DDA6E0DA
:10F90600C2DDACE0C0DDA1E0BEDDA5E3B7E0A3DD6E
:10F91600A0DC1E2FA0ECB7DD103021F4A0E4B7E088
:10F926009ADD04C0ABE4B7E096DDFFCF3324442470
:10F9360055246624E0E2F0E05E166F0644F40E9469
:10F94600C57E14F00E94CE7E0E94D57E99F7289837
:10F95600299A2A9ADFDD1E2F1530D1F4002450147F
:10F966006004ACF0E32DF42DB0973E2E4F2E00240C
:10F97600301440044CF4E0E0F2E03E2E4F2EE52D2C
:10F98600F62D31975E2E6F2E0E94D57E39F732C046
:10F99600133071F4E0E2F0E05E166F0644F40E9464
:10F9A600C57E14F00E94CE7E0E94D57E99F722C0B5
:10F9B600193001F50E94A07E0E94DE7E0E94907E94
:10F9C6000E94E17E0E946A7F0E94777F0E94DE7E0F
:10F9D6000E94947E0E94E17E0E948B7E0E94DE7EC3
:10F9E6000E94E17EF2DB08D0A8E8B3E10E94237F03
:10F9F6000C940000AFCFFFCF66971A930A93289A0C
:10FA0600299A2A98EFEFFFEFE0936407F0936507D2
:10FA1600E0911605E03011F00C94297E10E0A091DB
:10FA26001605A03011F41A3309F403C05BDE1E2F4D
:10FA3600F6CFE0911605E030A1F400E0053020F4A1
:10FA46000E94E47E0F5FFACF0E94ED7E0E94F47E54
:10FA5600E0936607F09367070E94F87E0E94FD7E9A
:10FA660001C0F4C0E0911605E030E9F43BDEEB8B13
:10FA760039DEEC8B0E94ED7EE0E0EF8BA4ED03DD3A
:10FA8600DE015396E8DC0E94F47EE0936207F09371
:10FA960063070E94027FF0700E94077FE091630770
:10FAA600F0700E94077FE0911605E03089F400E0CF
:10FAB600053020F40E94E47E0F5FFACF0E94ED7EAF
:10FAC6000E94F47EE0936807F09369070E94077F1F
:10FAD60000E00E940E7FF0F4E0911605E030C1F4DC
:10FAE600E0E0EB8BEC8B0E94ED7EE0E0EF8B0E947A
:10FAF600147FEA0FFB1FFF93EF930E94F47EAF91F2
:10FB0600BF91EC930E94147F0E94197F0E94077F89
:10FB16000F5FDFCFE0911605E03079F400E00530A5
:10FB260020F40E94E47E0F5FFACF0E94ED7E0E94D1
:10FB3600F47EE0936A07F0936B07E0916C07F0910F
:10FB46006D07F070A0E0B0E0AE1BBF0BA0936C0792
:10FB5600B0936D07E0916D07E070E0936D07E0915B
:10FB66006C07F0916D07A0916A07B0916B07EA17D1
:10FB7600FB0711F00C94287EA0916807B0916907E5
:10FB8600119729F40E941E7F0E944D7E5EC0A091AF
:10FB96006807B0916907129709F457C000E00E9400
:10FBA6000E7F10F00C94287E0E94147F0E94197F0D
:10FBB600E0936007F0936107E02FF0E03196DE01F5
:10FBC6001296AE0FBF1FEC91FE2FE0E0A0916007EA
:10FBD600B0916107EA0FFB1FE0936007F09361079E
:10FBE600E0916407F0916507E070DF010E94027FF3
:10FBF600E070EA17FB07A9F00E941E7FAF3FEFEF08
:10FC0600BE0721F00E941E7F0E944D7EA0916207D2
:10FC1600B091630731D00E94027FE0936407F093AE
:10FC26006507E0916007F0916107FA93EA93A09166
:10FC36006207B091630711D00E94027F3296E0936B
:10FC46006207F09363070E5FAACFE2CE2898299A3F
:10FC56002A9A1981088168960895BA93AA930F93F0
:10FC66001F93E881F9810A801B8011E00E94687E5B
:10FC76001F910F9124960895BA93AA93E881F9816A
:10FC86000F931F9313E00E94687E0E946F7E1F9160
:10FC96000F910DC0BA93AA93E881F9810F931F9330
:10FCA60015E00E94687E0E946F7E1F910F9122963A
:10FCB60008950F931F930FEE002E19E00E94687EA1
:10FCC6000E946F7E1F910F91089507B700FD0C9457
:10FCD600687E17BFE895089507B706FF089511E1F6
:10FCE600F4DFFACFEE81FF81688579850895A1E07A
:10FCF600B0E00C94237FE0935F07E6B1EF70A0912C
:10FD06005F07EA2BE0935F07E8B95F9A0C94147AD1
:10FD1600662777270E942D7F0895E0910105F0E080
:10FD26000895E0910605F09107050895E0E0F0E0FA
:10FD3600E0931005F09311050895E0911205F091F6
:10FD460013053297662777270895E983FA836B832D
:10FD56007C830895A981BA818B819C810895D901FC
:10FD6600EE27A50FBE1FAC910895E52FF0E0E20F38
:10FD7600F31FDF01EC910895D901EE27A50FBE1FF1
:10FD8600EC910895E0E2F0E03E0E4F1EE0E0F2E076
:10FD96003E164F06089533244424E1E0F0E05E0E5B
:10FDA6006F1E08956A925A92A32DB42D0E94A37ACB
:10FDB6001E2F103008950E94D67F08950E94D17F8D
:10FDC6000895E02FF0E0DE015396AE0FBF1FE0E08E
:10FDD600EC9308950E94757BED8B0E94757BEE8BEC
:10FDE6000895DE0153960C94047CE0916607F09129
:10FDF60067070895E0936C07F0936D070895E09107
:10FE06006207F09163070895A0916C07B0916D07A2
:10FE1600EA0FFB1FEFCFE9DFA02FB0E0AE17BF0759
:10FE26000895E02FF0E0DE0112960895AE0FBF1F91
:10FE3600EC91F0E00895A0916407B09165070895EC
:10FE4600109639F080EA9FE00197F1F7A89511978F
:10FE5600C9F70895EA0FFB1F681F791F0895AE0FB3
:10FE6600BF1F861F971F0895F195E195F0400895ED
:10FE7600EE230E2EFD01BC0131F0EE0FFF1F661FB3
:10FE8600771F0A94D1F70895EE230E2EFD01BC01CB
:10FE960031F076956795F795E7950A94D1F7089529
:10FEA600EE0FFF1FEE0FFF1FEE0FFF1FEE0FFF1FE0
:10FEB6000895F595E795F595E795F595E795F59503
:10FEC600E7950895E62FF72F60E070E008956F2F0D
:10FED600660F660B762F0895FA9FF02DEB9FF00DB7
:10FEE600EA9FE02DF10D08957A9F702D6B9F700D9E
:10FEF600F89F700DE99F700D6A9F602D710DFB9F35
:10FF0600600D711DE89F600D711D8827FA9FF02D09
:10FF1600610D781FEB9FF00D611D781FEA9FE02DA4
:10FF2600F10D681F781F08950024112490E1AA0F8F
:10FF3600BB1F001C111C0E1A1F0A18F40E0E1F1EE2
:10FF460001C0A1609A9599F7FD01D001089504D0EA
:10FF5600EBDF0EF489DF0895E894F7FF02C084DF33
:10FF66006894B7FF06C0A095B095119600F8039463
:10FF760000FA0895ED91FC9111970895ED91FD9188
:10FF86006D917C9113970895ED91FD916D917D9101
:10FF960008957E936E93FE93EE930895A881B9819A
:10FFA6008A819B810895E883F9836A837B83089518
:10FFB6009A938A93BA93AA930895EA17FB07680758
:10FFC600790708955A934A933A932A931A930A9370
:10FFD60008955D814C813B812A81198108810895AC
:00000001FF
